:020000040000FA
:06000000020A08022003C1
:03000B0002200BC5
:03001300022013B5
:03001B0002201BA5
:0300230002202395
:03002B0002202B85
:0300330002203375
:03003B0002203B65
:0300430002204355
:03004B0002204B45
:0300530002205335
:03005B0002205B25
:0300630002206315
:03006B0002206B05
:03007300022073F5
:03007B0002207BE5
:03008300022083D5
:03008B0002208BC5
:03009300022093B5
:03009B0002209BA5
:0300A3000220A395
:0300AB000220AB85
:1000B3000220B3E590540C23C0E0740EC0E0C0826C
:1000C300C083020E00E590540C23C0E0740EC0E020
:1000D300C082C083020E08E590540C23C0E0740E66
:1000E300C0E0C082C083020E10E590540C23C0E030
:1000F300740EC0E0C082C083020E18EFC403900EDA
:02010300007387
:10010600E56A245EF8E6056A22785B300702785EC7
:10011600E475F0011206DD0206482000EB7F2ED2C0
:10012600008018EF540F2490D43440D4FF30040BD1
:10013600EF24BFB41A0050032461FFE56B6002157B
:100146006B056EE56E7002056D30070D785BE47524
:10015600F0011206DDEF0206CB020D387403D2075A
:100166008003E4C207F56A8B5B8A5C895DE4F56B04
:10017600F56DF56EE56B60077F2012014180F57520
:100186006CFFC201C200C202C203C205C206C20897
:1001960012010FFF700D3007057F00120152AF6E7E
:1001A600AE6D22B4255FC2D5C20412010FFF24D062
:1001B600B40A00501A75F00A786B30D50508B6FFF8
:1001C6000106C6A426F620D5047002D20380D924DF
:1001D600CFB41A00EF5004C2E5D204020352D20192
:1001E60080C6D20080C0D20280BCD2D580BAD205E9
:1001F60080B47F201201412002077401B56B0040D4
:10020600F1120106FF12014102017AD208D20680DC
:1002160095120106FB120106FA120106F94A4B7005
:100226000679237A047BFF20022EE56B602A7E0086
:100236008E8275830012069E60060EEE656C70F067
:10024600C2D5EBC0E0EAC0E0E9C0E0EE120399D007
:10025600E0F9D0E0FAD0E0FB120648FF60AAEBC056
:10026600E0EAC0E0E9C0E0120141D0E02401F9D0A3
:10027600E03400FAD0E0FBE56C0460DCD56CD98094
:10028600877BFF7A037995D202809C791080027968
:1002960008C206C2088008D2D5790A8004790AC243
:1002A600D5E56C047002F56CE4FAFDFEFF1201065A
:1002B600FC7B08200113120106FD7B1030000A1298
:1002C6000106FE120106FF7B20EC3382D592D55043
:1002D60013C3E43000069FFFE49EFEE42001039D65
:1002E600FDE49CFCE4CBF8C201EC700CCFCECDCC87
:1002F600E824F8F870F38017C3EF33FFEE33FEED12
:1003060033FDEC33FCEB33FB994002FB0FD8E9EBF2
:10031600300105F8D0E0C448B201C0E00AEC4D4E09
:100326004F78207B0070C2EAB56C0040BCC0E0127A
:10033600039BD0F0D0E0200104C4C0E0C4B201C0E9
:10034600F012012AD0F0D5F0EB02017A1206ED0286
:10035600175302915801E84C01E44202954F029D61
:1003660044029D4901FD4302A35502874602874583
:1003760002874704435001EC2D01F02E02132B0196
:10038600F423021120042C2A01AC480000020B3F82
:100396003F3F00790AA2D5200314300509B910029F
:1003A6000404B9080104A2D5200602500104200263
:1003B600689202B56B005034C0E07F203003197F8D
:1003C60030A20272067205500F1203F2C202C20672
:1003D600C205C2087F30800F300503E9C0E0120174
:1003E60041300503D0E0F9D0E0B56BCC3005177F7E
:1003F60030B9100C1201417F583004077F78800312
:10040600B908031201413002057F2D0201417F2008
:100416002008F87F2B2006F322920280CF286E75E3
:100426006C6C2900D2011201063001F8C201786B0A
:1004360030D50108F60201AC2D5043495812010689
:100446002403B405004001E490043E931201327483
:100456003A120132D203756B04020291E4F556F5A5
:1004660057F558E5097015120D687BFF7A0F794F1D
:100476001201687BFF7A0F798102058D120D687A69
:100486000F799612063F120D4C8F31BF3AF8120DB6
:10049600008F4B120D00E48F50F54FF54EF54D12BF
:1004A6000CC878081206858F508E4F8D4E8C4D12D3
:1004B6000D00E5504FF550E54FF54FE54EF54EE58D
:1004C6004DF54D120D008F4CE4F52FF530120CCF83
:1004D6005014120D0074322530F8A6070530E530A9
:1004E60070EB052F80E7120D008F55E4FF7E20FD8F
:1004F600FCAB50AA4FA94EA84DC312066150030289
:100506000593D3E54C9401748094804003020593CF
:100516007B007A007932756200854B63120CC61235
:100526000A94B297E4F556F52FF530120CCF502405
:10053600E5302550FFE52F354FFEE4354EFDE43519
:100546004DFC120B6BEF2556F5560530E53070DB8A
:10055600052F80D7E54B2556F556120CC67808129E
:100566000672EF2556F556E550FFEF2556F556254A
:100576004CF5562555F556FF3395E04F600F120D95
:10058600687BFF7A0F79AC120168020D71120D6853
:100596007A0F79CB12063FE54C6401600302048CA6
:1005A600F52FF5300530E5307002052FB410F5E56E
:1005B6002FB427F0750801120D687BFF7A0F79CEEC
:1005C6001201687BFF7A0F79F0120168120D71E44F
:1005D600F557F558F554755320F552F551AB54AA15
:1005E60053A952A851120CA9502CAF54AE53AD5278
:1005F600AC51120B6BEF2558F558E43557F557E516
:10060600542401F554E43553F553E43552F552E4D8
:100616003551F55180C7C3E49558F55AE49557F519
:1006260059FF3395E08F6C120CBD1208EC855A6C9D
:100636007FFF120CBF1208EC227BFF120168120D1D
:100646007122BB010689828A83E0225002E722BB1F
:10065600FE02E32289828A83E49322EB9FF5F0EA85
:100666009E42F0E99D42F0E89C45F022E8600FECDE
:10067600C313FCED13FDEE13FEEF13FFD8F122E8D2
:10068600600FEFC333FFEE33FEED33FDEC33FCD8E2
:10069600F1228A838982E473BB010CE58229F58203
:1006A600E5833AF583E0225006E92582F8E622BB87
:1006B600FE06E92582F8E222E58229F582E5833AFB
:1006C600F583E49322BB010689828A83F0225002D5
:1006D600F722BBFE01F322FAE6FB0808E6F925F04D
:1006E600F618E6CA3AF622D083D082F8E49370125E
:1006F600740193700DA3A393F8740193F582888314
:10070600E4737402936860EFA3A3A380DF85EF26EA
:10071600E4F5A753D9BF120D5D120C47E4FF120C86
:1007260079C2AFD297752BFF752C20752D00E4F595
:1007360022F523F52A752920F528F527AB2AAA29BB
:10074600A928A827120CA9502CAF2AAE29AD28AC8F
:1007560027120B6BEF2523F523E43522F522E52A34
:100766002401F52AE43529F529E43528F528E43568
:1007760027F52780C7120CBD120B6BEF752500F508
:10078600247FFF120CBF120B6BEF2525F525E435F0
:1007960024F524C297E5252523F523E5243522F5FE
:1007A6002245236003020855AA2CA92D1206982279
:1007B6007E80AB36AA35A934A833C30206617E8093
:1007C600AB6BAA6AA969A868C3020661E536F53665
:1007D600E5354480F535E534F534E533F5338535CF
:1007E6003985363A53F5CF22E56BF56BE56A4480D9
:1007F600F56AE569F569E568F568856A6F856B7080
:1008060053F5CF22E55EF55EE55D4480F55DE55C7A
:10081600F55CE55BF55B855D61855E6253F5CF2230
:100826007E80AB5EAA5DA95CA85BC3020661C2AF0F
:10083600E4F5A7FFFDFC22E4FFFE7D01FC227F001C
:100846007D017C002275EF0275B7A575B7F12212FE
:100856000D217F01120C791208E5120D71120D4C53
:100866008F2EE52E24CF601614602524F3603024E5
:100876003770311208D2120D4C1208D28021120B99
:1008860000120D687A0E791C1208DC1204628026AA
:10089600120D687A0E79371208DC75EF1080171280
:1008A60008E5800F120D68120C117BFF7A0E794B4A
:1008B600120168120D71120D687BFF7A0E796212B1
:1008C6000168120D71120D4C8F2E8096120D4C126E
:1008D6000D4C120D4C227BFF120168120D71221273
:1008E6000D68120C11228F6B8E6A8D698C6885A734
:1008F6006DA2AF920085F56E1208341207C450053A
:10090600120800802612083D1207C650081207EE8C
:1009160043F51080161208441207C450081207EE59
:1009260043F520800612080043F530E4F5EF75FF25
:10093600A0FFEFC394FF7480948050030F80F3E50B
:10094600FF20E6037F002212084B438F0175FFA0AC
:1009560075EF02857082856F83E56CF0E4F5EF75BF
:10096600FF8075EF02538FFE856EF5856DA7A20099
:1009760092AF7F01228F368E358D348C3385A73723
:10098600A2AF920085F5381208341207B650051248
:1009960007E4802612083D1207B850081207D24312
:1009A600F51080161208441207B650081207D243F3
:1009B600F52080061207E443F530E4F5EF75FFA055
:1009C600FFEFC394FF7480948050030F80F3E5FF1C
:1009D60020E6037F002212084B438F0375FFA075A4
:1009E600EF02853A82853983E4F0F5EF75FF80756D
:1009F600EF02538FFC8538F58537A7A20092AF7FAB
:100A06000122787FE4F6D8FD758170020A4F02074D
:100A160013E493A3F8E493A34003F68001F208DFFE
:100A2600F48029E493A3F85407240CC8C333C454B0
:100A36000F4420C8834004F456800146F6DFE48064
:100A46000B0102040810204080900D7AE47E019389
:100A560060BCA3FF543F30E509541FFEE493A36036
:100A6600010ECF54C025E060A840B8E493A3FAE491
:100A760093A3F8E493A3C8C582C8CAC583CAF0A3E2
:100A8600C8C582C8CAC583CADFE9DEE780BE8F5EF5
:100A96008E5D8D5C8C5B8B5F8A6089618F678E66ED
:100AA6008D658C64E563255EFFE562355DFEE435A4
:100AB6005CFDE4355BFCAB67AA66A965A864C31256
:100AC60006615035AF67AE66AD65AC64AB5F056178
:100AD600E561AA607002056014F9120648F56C1209
:100AE60008ECE5672401F567E43566F566E43565E7
:100AF600F565E43564F56480AB22120D687BFF7AF8
:100B06000F791B120168120D71E4F532753120F56B
:100B160030F52FE47FFF7EFFFDFCAB32AA31A93012
:100B2600A82FC31206615022AF32AE31AD30AC2FC2
:100B360012097BE42532F532E5313402F531E4352C
:100B460030F530E4352FF52F80C9E42532FFE53145
:100B56003402FEE43530FDE4352FFC12097BE4F562
:100B660008750901228F5E8E5D8D5C8C5B85A75FA3
:100B7600A2AF920085F560120834120826500512BD
:100B8600081C802612083D120828500812080A433D
:100B9600F5108016120844120826500812080A4357
:100BA600F520800612081C43F53085628285618334
:100BB600E493FF8560F5855FA7A20092AF228F5E62
:100BC6008E5D8D5C8C5BE4F562F561F560F55FAF7B
:100BD6005EAE5DAD5CAC5BAB62AA61A960A85FC3AB
:100BE6001206615025E4FFFE0FBF00010EBE04F899
:100BF600BF38F5E5622401F562E43561F561E43557
:100C060060F560E4355FF55F80C5227A0E7977126C
:100C16000C3F7A0E79951201687A0E79A2120C3F72
:100C26007A0E79C51201687BFF7A0E79E91201689E
:100C36007BFF7A0F79040201687BFF1201687BFF54
:100C460022AFA775A70F75F1F875F30375F4F8755C
:100C5600A41075A59575A60375AE7875AF0375D402
:100C6600CF75E10175C742E4F5B575B00775A0FC0F
:100C76008FA7228F2F85A73075A70FC2B3E52F2424
:100C8600FF92B4C2B6C2A0C2A17F0A120CB6120B62
:100C9600C4E52F24FF92B57F32120CB6120BC48521
:100CA60030A722E47FFE7EFFFDFCC30206617F01C2
:100CB6007E007D007C00227FFE7EFF7D007C002280
:100CC600AF50AE4FAD4EAC4D22C3E530954BE52F40
:100CD600940022EF7E0024D0B40A00401B24F9B40D
:100CE6000A004011B41000400F24E0B40A00400589
:100CF600B41000400374FFFEFF22120D4C8F5C12ED
:100D06000D4C8F5DAF5C120CD9EFC454F0F55BAFA0
:100D16005D120CD9EF255BF55BFF22AFA7E4F5A7C3
:100D260075981075A70F75ACF075ADFF75AB438F51
:100D3600A722AEA7E4F5A7BF0A027F0D8F993099C7
:100D4600FDC2998EA722AFA7E4F5A73098FDAE990C
:100D5600C2988FA7AF0622AFA775A70F75A1C78F39
:100D6600A72243B501120CB4020BC453B5FE120CF4
:0B0D7600B4020BC401090001080000DA
:040E00005390F322F6
:070E080043900C5390F72208
:070E100043900C5390FB22FC
:100E180043900C220A2A2A2A20466C6173682070A3
:100E280061676573206572617365642E0A20000A24
:100E38002A2A20524553455454494E47202A2A0A03
:100E48000A20000A2A2A2A20556E6B6E6F776E20B8
:100E5800436F6D6D616E640A20000A456E74657299
:100E6800206120636F6D6D616E64203E0A20000A68
:100E78000A433830353146353830204669726D7747
:100E880061726520557064617465720A004C6F6107
:100E98006465725F76362E330A002D2D2D2D2D2D8B
:100EA8002D2D2D2D2D2D2D2D2D2D2D2D2D2D2D2D6A
:100EB8002D2D2D2D2D2D2D2D2D2D2D0A00312E20B2
:100EC800457261736520464C41534820616E642029
:100ED800557064617465204669726D776172650A40
:100EE80000322E2043616E63656C204669726D770F
:100EF800617265205570646174650A003F2E205048
:100F080072696E7420436F6D6D616E64204C6973F5
:100F1800740A000A2A2A2A2045726173696E6720BA
:100F2800666C6173682066726F6D2030783130307E
:100F38003020746F20307830464646462062616E15
:100F48006B7320302C31000A2A2A2A204174206C25
:100F580065617374206F6E6520464C41534820705C
:100F6800616765206D7573742062652065726173B1
:100F78006564207072696F720020746F20746869EC
:100F880073206F7065726174696F6E2E0A000A5261
:100F98006561647920746F20726563656976652E72
:100FA8002E2E0A002A2A2A20436865636B73756D02
:100FB800206661696C65642C2074727920616761B0
:100FC800696E006F6B000A2A2A204669726D776184
:100FD80072652055706461746520436F6D706C652F
:100FE80074652E202A2A0A000A506C656173652CE4
:090FF8002072657365742E0A0075
:00000001FF
